:100000007FC0A3C0A2C0A1C0A0C0ADC09EC09DC003
:100010009CC09BC09AC099C098C097C096C07445B8
:1000200079467D47824887498B60906194629963E5
:100030009D64A265A766AB67B068B469B980BE81EC
:10004000C282C783CB84D084D484FF2103030405F8
:1000500006080A0C0F13171C21282F373F49545F3D
:100060006C7A8999ABBED2E8FFFFFFFFFFFFFFFF6D
:10007000FFFFFFFFFFFFFFFFFFFFFFFFFFFFFFFF90
:10008000FFFFFFFFFFFFFFFFFFFFFF00000000007B
:100090000000000000000000000000000000000060
:1000A0000000000000000000000205080B0E121600
:1000B0001A1E22272C31363B41474D545B62697131
:1000C000798189929BA4AEB8C2CDD8FF40000B4085
:1000D000000B2340000B1A2E40000B172432400067
:1000E0000B141F293540001D40F200F3F40B1D4096
:1000F0000009121D2E40000B1D3200F3F4F24000E7
:1001000011241FBECFE5D1E0DEBFCDBF20E0A0E6C9
:10011000B0E001C01D92A737B207E1F7E8E7F0E0D1
:1001200085E5808781E08383148212828683118231
:1001300085E081878FE48287E1E6F0E08DEF8783B9
:100140008EEF8583712CC7D0BFC25ACF815090E00B
:10015000FC01E45BFF4FE491E9BDFC01E457FF4F74
:10016000849188BD0895189525B7277E25BF29B7A6
:10017000226029BF21E022BF019728F020E1889565
:100180002150E9F7F9CF089588EE93E0EDCF369A44
:100190003699FECF85B10895CF93C72D81E0870DA5
:1001A0008F73782E662D90E081D26FEF8C2F90E0C8
:1001B000CF917CC2FF920F931F93CF93DF93F82EC2
:1001C00009E710E0CEE7D0E0F11005C0CE0166D21D
:1001D000F801808304C0F8016081CE0167D22197C5
:1001E0000F5F1F4FC437D10579F7DF91CF911F9172
:1001F0000F91FF900895D0DF81E0DCCF811103C023
:1002000019BC18BC0895A2CFCF93DF93D82F90913B
:1002100060002D2F291BC1E009F4C0E0259525952C
:10022000C22BC90FC09360008C2FE8DF83E090E001
:100230009BDFDC13ECCFDF91CF9108950F931F93D9
:10024000CF93C82F8B01CC2361F081E17FDFC80100
:100250008BDF19BC18BCC80187DFC80185DFC1501E
:10026000F2CFCF911F910F910895EF92FF920F93CC
:100270001F93CF93C8E0E82EF12C062F10E080E406
:1002800065DFC70171DF19BC18BCC8016DDFC15043
:10029000B1F7CF911F910F91FF90EF9008951F93A9
:1002A000CF93DF938FEA87B986EC86B910E1C0E07F
:1002B000D0E085E090E058DF6ADFC80FD11D115013
:1002C000C1F7CE0124E0969587952A95E1F7DF9155
:1002D000CF911F9108951092770083EA87B986EC39
:1002E00086B93699FECF369A3699FECF85B180957C
:1002F000582E87E790E0D2D1853519F0612C7BDF4D
:1003000011C0712C872D90E0C9D1682E8F3F19F054
:1003100080E050DF07C0872D91E0970D792E803463
:1003200088F3F6CF20918100C0917B0010917C0072
:1003300080917900882319F010E0C0E029E02F5F58
:1003400090E040E050E0ACECB0E0222379F0BD0159
:100350006F5F7F4FFB013197E491EE2319F0962FE9
:100360009A1BF6CF2150AD01DB01EFCF092F6C2F87
:1003700070E0A92FB0E0E02FF0E0112321F09D0103
:100380002E1B3F0B05C09F0121503109260F371F3F
:100390003197E40FF51FF49026593F4FF901F08291
:1003A000015049F79C0F90938300CC2371F01123E7
:1003B00029F0292F30E02150310902C020E030E03F
:1003C000F901E659FF4F41E0408324E0290F322F25
:1003D0003150E32FE91BF0E0E550FF4FE491A32FEC
:1003E000B0E0A659BF4FEC933913F2CFE22FF0E003
:1003F000E759FF4F31E050916A004081541330E0DB
:10040000231B20938400362D353FE8F5452D4134DC
:10041000B0F4809185008F3F29F48091770080931C
:10042000850006C081E0860D682E891708F0612CD2
:10043000809185008F5F8F718093850024C03091FB
:100440007700309385004F3AC0F430917E0033231B
:1004500011F0882339F081E0860D682E891798F015
:10046000612C11C0862D6916D9F3662019F08150D0
:10047000682E09C02150622E06C08111F1CF8091F3
:100480007A00882369F38FE384BB8BE087BB88EF16
:1004900088BB81E083BF91EA9ABD85B7806285BF42
:1004A000789497B986EC86B9C62DC53F10F0612CBB
:1004B0003CC080918500803138F4E62DF0E0E659AB
:1004C000FF4FC081DC2F31C05FDE809177008093C9
:1004D0008500C9E7D0E000E010E0FF24F39481E05C
:1004E000800F0F5F1F4F98819F3F29F4219608309E
:1004F0001105A9F7E2CF6DE570E0A0DEF801EF5934
:10050000FF4F608088818F25888375DE6FE070E003
:1005100080E294DE88818F258883612C6CDE34DE56
:1005200080917900882311F3C8CF36DE10E0F12CDA
:1005300081EAE82E96ECD92ECC24CA94C23F39F435
:1005400068E284E192DE60E588E28FDE66C0C33F48
:1005500081F404E080E4FADD85E090E005DE8DE1E1
:10056000F5DD81E490E000DE0150A1F780ED92E03E
:1005700053C0C43F51F584E690E0F6DD08DE90E01C
:10058000292F30E0F901E25EFF4FE491E81710F403
:100590009E5FF6CFF901E15EFF4F04916DE770E0D9
:1005A000802F82958695877049DE8EEE92E0DCDDA5
:1005B00065E070E081E042DE85E694E0D5DD6DE740
:1005C00070E0802F8F713ADE0DC0CE3F71F400E0F5
:1005D0000093810010DE6AEF70E081E02FDE0F5F94
:1005E0000930B1F7D1DDD0DD18C0CD3F39F58FEF3F
:1005F0008093820000DE80E107DEC6DDC5DD80E499
:1006000003DE4DDE80938200F6DDBEDDBDDDF9CF79
:10061000D132F8F484EF91E0A7DD809177008093E8
:100620008500B5DD823808F037C01F5F183008F448
:1006300085CFD134A8F010E0D0E2C0E28D2FE4DD08
:100640002EDEE7B8D6B8F39490918200891710F3A4
:10065000DFCFF4E1FF15F0F6C0927700D0E2DACFF9
:10066000D23030F08D2F86958695D695D80F13C051
:1006700019BC18BC85B7877E806185BFF89485B7A3
:10068000846885BF8B7F85BF85B7806285BF88956D
:1006900085B78F7D85BFCD2F10E050CFE199FECF7C
:1006A0001FBA8EBBE09A99278DB30895262FE19942
:1006B000FECF1CBA1FBA8EBB2DBB0FB6F894E29AC0
:0C06C000E19A0FBE01960895F894FFCF58
:00000001FF
